:020000040800F2
:102000002808002071410008AB320008B9320008EE
:1020100000000000000000000000000000000000C0
:10202000000000000000000000000000BD320008B9
:102030000000000000000000BF320008AD320008C0
:10204000E72F00080000000027300008733E00085A
:102050000F4100081B410008954100089741000806
:102060000000000099410008FD2200089B41000883
:102070009D4100089F410008A141000800000000A8
:10208000A3410008A541000800000000A741000886
:10209000A9410008AB410008AD410008AF4100086C
:1020A000B1410008B3410008B5410008B74100083C
:1020B000B94100080121C006C00E8140B44801604A
:1020C000704700B5BFF34F8FB248B3490860BFF304
:1020D0004F8F00BFFDE780B588B00020AF49087082
:1020E000072000F026FE002000F023FE002301223E
:1020F0000B219020C00500F0CBFE00230122082117
:102100009020C00500F0C4FE01220B219020C005E4
:1021100000F057FF012208219020C00500F051FF78
:10212000012000900323022209219020C00500F025
:10213000E8FE01200090032302220A219020C0051E
:1021400000F0DFFE9649974800F04EFF954800F0FA
:1021500065FF102001900020029080200390002055
:10216000049000200590002006900020079001A90F
:10217000B34800F059FF0020019000200290802019
:1021800003900020049000200590002006908020FD
:102190008001079001A9AB4800F046FF01210A2009
:1021A00000F06EFF0A20FFF785FF01210A2000F0F2
:1021B00067FF0A20FFF77EFFC9480078012101432D
:1021C000C7480170C6480078EF210140C44801703B
:1021D000C3480078FB210140C1480170C048007825
:1021E000F7210140BE48017009B000BD80B5BC4870
:1021F00000780100C907C90F00294CD000F0FEFF8C
:1022000001280BD1B648007804210143B44801707D
:10221000B348007808210143B14801708A4800782A
:1022200000282ED101F000F888490860AC480078F9
:10223000C0B240090100C907C90F002902D000201F
:102240005649087055480078012802D100F008FA74
:1022500027E052480078022802D100F085FA20E0F9
:102260004E480078002802D100F040F919E09C485F
:102270000078102101439A480170002047490870F6
:102280000FE000F0D1FF71490968401A1F2808D3F8
:10229000FFF717FF05E092480078102101439048AE
:1022A000017001BD00B5010000200A00D2B2002A71
:1022B0000AD18B490978C9B209090A00D207D20F9D
:1022C000002A10D001200EE0C9B202290AD18449A7
:1022D0000978C9B249090A00D207D20F002A02D0F0
:1022E000012000E00020C0B200BD7D480078010060
:1022F000C9B2C9080800C007C00F704780B552486E
:102300000078012827D177480068202108407549C6
:102310000860002812D0744800684006FBD5484881
:1023200000680221884346490860C54800682021AA
:102330000143C348016000F08BF828E04048006882
:10234000082188433E490860BD4800688021014358
:10235000BB4801601BE03A480068082188433849BF
:102360000860374800680221884335490860B4484E
:102370000068802109010143B1480160B04800684C
:10238000802189000143AE48016000F061F801BD81
:1023900000E100E00400FA050CED00E01E0400205E
:1023A000810600000038014010B5040001202649D4
:1023B000087001220B219020C00500F002FE0122CE
:1023C00008219020C00500F0FCFD002003E0002162
:1023D0009C4A1154401CFF28F9D919480068012172
:1023E0008843174908601748006801218843154948
:1023F0000860954804609548954908609548964955
:1024000008600F480068022101430D4801600C4834
:102410000068082101430A48016090480068402193
:1024200001438E48016006480068012101430448C9
:102430000160C348006880210143C148016010BDAC
:102440001C000240300002401D040020E003002078
:1024500080B50020BB490870002208219020C005EB
:1024600000F0AFFD00220B219020C00500F0A9FD77
:10247000002003E00021734A1154401CFF28F9D9C1
:10248000B148006801218843AF490860AF4800683F
:1024900001218843AD49086080204000AC490860B4
:1024A000AC48AD4908606748AC490860A748006877
:1024B00002210143A5480160A448006808210143A6
:1024C000A2480160A1480068012101439F480160C2
:1024D0009B480068402101439948016001BD00000C
:1024E0001C040020000002401C38014080B59C48BC
:1024F0000078C0B240080100C907C90F002969D19E
:1025000029209849087000209649487088209549EC
:1025100088704B209349C870532092490871452018
:102520009049487156208F4988714F208D49C87154
:1025300000208C49087200208A494872002089498D
:10254000887200208749C8720020864908730020DD
:102550008449487300208349887300208149C873E7
:1025600000208049087400207E49487400207D497D
:102570008874FF207B49C874FF207A490875FF20C2
:102580007849487589207749887576207549C875D6
:10259000002004E0FF21734A12181176401C132812
:1025A000F8D33120B14908703020B149087000F0EB
:1025B00065F9B0490860AF480068FFF7F5FE684864
:1025C0000078022101436648017000F02DFEAA49FF
:1025D000086034E000F09EF9012829D1CB4840780A
:1025E000BB2802D1FFF76DFD29E0C8488078882814
:1025F00016D1C648807DC549CA7DFF21C943114314
:10260000CA43904209D100F086FE012802D1012080
:10261000BF49087000F046FA11E000F029FA0EE018
:10262000F32802D1FFF74DFDFCE700F021FA06E0A8
:10263000022802D100F01CFA01E000F0F8F901BD17
:1026400004000240C8010020200002402838014058
:1026500024000240C8000020280002402038014029
:1026600080B53F480078C0B240080100C907C90FD3
:1026700000293AD10A203B490870002039494870A6
:1026800006203849887000203649C8700020C043B1
:1026900000F04DFF010E334A11710100090C314A5F
:1026A0005171010A2F4A91712E49C87100202D499C
:1026B000087200202B49487200202A4988720020A5
:1026C0002849C87200F0DAF86A4908606948006869
:1026D000FFF76AFE2248007802210143204801707A
:1026E00000F0A2FD6449086029E000F013F9012818
:1026F00023D186484078BB2802D1FFF7E2FC1EE0D8
:102700008248807886280DD1804800F0DEF90128C3
:1027100002D100F0C7F901E000F0AAF902207C49DB
:1027200008700CE0F92805D100207949087000F004
:10273000B9F904E000F09CF901E000F078F901BD7E
:10274000083801401D0400201C00024030000240F7
:102750003400024024380140380002403C0002406E
:102760001C0400204803002080B5CD480078C0B28A
:1027700040080100C907C90F002935D10720BB490E
:1027800008700020B94948705220B8498870332039
:10279000B649C8703120B54908713020B349487135
:1027A0003120B249887100F0CFFD0100AF4AD171EC
:1027B000C143AE480172BA480078FB210140B848D5
:1027C000017000F05BF82B4908602A480068FFF7A9
:1027D000EBFDB348007802210143B148017000F0DD
:1027E00023FD254908603FE000F094F8012839D125
:1027F00046484078BB2802D1FFF763FC34E04348E9
:102800008078F0281BD14148C078522814D101208B
:102810003F490870A2480078C0B280080100C9078B
:10282000C90F002905D19E480078F72101409C4836
:10283000017000F037F917E000F01AF914E0F928F8
:1028400005D100F02FF90020314908700CE08628EE
:1028500005D100F027F901202D49087004E000F0AF
:1028600007F901E000F0E3F801BD00006A03002071
:102870006B030020E4030020DC03002038B50125B1
:102880000220BB49087000241CE07848005DC0B2FB
:102890000009C0B200F06AFEB549022262438918FD
:1028A00048707248005D0007000F00F05FFEB049FD
:1028B0000222624389188870002C02D06B48005DA8
:1028C0002D18641C69480078401CA042DDD2E84302
:1028D000C5B2280900F04AFEA549022262438918C0
:1028E00048702807000F00F041FEA1490222624310
:1028F0008918887003209E49022262438918C87093
:1029000002204443241D200032BD0000C8020020E4
:102910001E040020F8B50020002200E0521CFF2A0F
:1029200007DC944B9B5C032BF8D111000023914CE6
:10293000A354FF2A6ADC4C1E00E0641E002C66D4FF
:102940008C4A125D022AF8D100208A4A10550D1BCC
:102950006D1C083D2000401CC0B20100491CC9B2DA
:10296000844A105C834A515CC9B2C0B200F051F88D
:1029700081490870E80708D46808001F792804D244
:1029800068087D490978884201D002203FE06F083D
:1029900001252000C01CC0B20100491CC9B2754A03
:1029A000105C744A515CC9B2C0B200F032F872498E
:1029B0004870714840782E1800251AE02000401D0C
:1029C000022169434018C0B20100491CC9B2694ADA
:1029D000105C684A515CC9B2C0B200F01AF866498E
:1029E00049198870BD4203D263484019807836186F
:1029F0006D1CAF42E2D2F043C0B25F49C919897879
:102A0000884201D0022000E0012000E00020C0B296
:102A1000F2BD38B50C000021C0B200F093FD0501F5
:102A20002000C0B200F08EFD2818C0B232BD80B5C3
:102A300000F0FAFB51490968401A652814D3504840
:102A40000068401C4E4908604D480068052805D3C1
:102A50001348007820210143114801701048007884
:102A6000FD2101400E48017001BD00004803002017
:102A700000B544480068401C42490860414800686D
:102A8000052805D306480078202101430448017039
:102A900003480078FD2101400148017000BD00009D
:102AA0001C040020002037490860002034490860D9
:102AB00035480078FD2101403348017032480078E4
:102AC000DF21014030480170704738B50400E07ED6
:102AD000227FFF21C9431143CA43904245D12A496D
:102AE0000978C9B2C9080A00D207D20F002A02D158
:102AF00000F038FC03E000F027FC00F033FCE07845
:102B00000006217909044018617909024018A17969
:102B1000401800F02DFC627A00231B06100A0343C4
:102B20001206A07A00210904050C2943000480182C
:102B30005941E27A00231B02150E2B431202121890
:102B40004B41207B002180185941627B00231302F6
:102B5000002212184B41607B0021010000208018E8
:102B6000594100F008FC012000E00020C0B232BD55
:102B7000C8000020C8010020C8020020DC0300209B
:102B8000E8030020EC0300201C04002080B500F0C6
:102B90000DF89D499D4A126812091207120F895CAF
:102BA000C8409B4908609A48006802BD10B50020E3
:102BB0000020002000200020944800680C210140E3
:102BC000042902D0082902D017E0924C16E092495D
:102BD000820C1207120F8C5C9049914A12681207FE
:102BE000120F895CC00305D58A4800F04AFD604396
:102BF000040001E08B48444300E0864C200010BDF7
:102C00008948006801210143874801607F480068C6
:102C1000864901407D48016083480068844901403D
:102C20008148016080480068824901407E48016017
:102C3000764800688049014074480160784800681F
:102C40000F218843764908607C4800681321884337
:102C50007A4908607A4800680100C907C90F7848B6
:102C60000160002077490860704700B56E48006831
:102C7000754901406C4801606B4800688001FBD4D5
:102C8000674800680F218843654908606448006808
:102C9000634908605D4800686C4901405B48016019
:102CA0005A480068A02189030143584801605E48E2
:102CB00000688021490401435B4801605A4800686C
:102CC0008001FBD562480068012101436048016032
:102CD0004E480068F02188434C4908604B48006822
:102CE0004A490860504800688001FBD547480068A1
:102CF0000321884345490860444800680221014394
:102D000042480160414800680C2101400829F9D17E
:102D10003E4800684F4901403C4801603B4800681C
:102D20003A4908604C480068012101434A48016063
:102D300000BD00B50100C9B2012907D147480068AC
:102D4000802189020143454801605CE00100C9B26D
:102D5000022907D1414800688021C90201433F4848
:102D6000016050E00100C9B2032907D13B48006867
:102D70008021090301433948016044E00100C9B2E0
:102D8000042907D1354800688021490301433348AD
:102D9000016038E00100C9B2052907D12F48006859
:102DA0008021C90301432D4801602CE00100C9B214
:102DB000062907D12A4800688021C9030143284811
:102DC000016020E00100C9B2072907D1244800684A
:102DD0008021C90101432248016014E00100C9B209
:102DE000002906D11D480068012101431B480160EC
:102DF00009E0C0B2082806D11948006880210901FD
:102E000001431748016000BD304100080410024032
:102E1000C400002000127A00404100085041000820
:102E20002C10024000093D00001002400CB8FF00C9
:102E3000FFFFF6FEFFFFFBFFFFFFC0FF3010024069
:102E40003410024008100240FFFFFFFEFFFFC2FFE8
:102E500000200240FFF8FFFF0C1002401410024057
:102E60001810024030B40368032402254D43AC40DF
:102E7000A3430360C368032402254D43AC40A3432E
:102E8000D2B2022461438A401A43C26030BC704708
:102E900070B50468032502264E43B540AC430125B6
:102EA00002264E43B540254305608468032502266B
:102EB0004E43B540AC43DBB202254D43AB40234308
:102EC0008360436801248C40A343112A10D101225E
:102ED0008A401A434260C268032302244C43A34041
:102EE0009A430123022461438B401343C36007E0EC
:102EF0004360C2680323022461438B409A43C2604B
:102F000070BDF0B5059C0D00EDB2082D0BDA056A19
:102F10000F2604274F43BE40B54304264E43B4401A
:102F20002C43046210E0466A0F27BC460D00083DA2
:102F300004277D436746AF40BE430D00083D04278C
:102F40007D43AC40344344620468032502264E436B
:102F5000B540AC43022502264E43B54025430560EB
:102F60008468032502264E43B540AC43DBB20225FC
:102F70004D43AB4023438360436801248C40A3430B
:102F8000122A10D101228A401A434260C2680323E8
:102F900002244C43A3409A430123022461438B4003
:102FA0001343C3600CE04360C268032302244C4314
:102FB000A3409A430123022461438B401343C3601F
:102FC000F0BD00B5D2B2002A03D001228A4082614E
:102FD00003E0012210318A40826100BD02690120B4
:102FE000884010407047FEE7002202600268084BEC
:102FF000134303604268074B13404360C16041685C
:10300000054A0A40426081682A22914381607047E4
:103010000C800000FFCFFFFFFFB7FFFF0168012218
:103020000A4302607047FEE710B4026801239A4326
:1030300002600368094A1A400B684C681C438B689D
:103040002343CC681C430B6923434C691C438969A7
:1030500021431143016010BC704700BF0FC0FFFF48
:1030600080B5401E2949086000210020C04300F0BF
:1030700007F800202649086007202649086001BD9E
:10308000F0B5020052B2002A23D5234B020052B2FF
:103090001207120F083A9208042462431E4C0500DE
:1030A0006DB22D072D0F083DAD08042675436459F8
:1030B000FF258607B60F08277E43B540AC4389013C
:1030C000C9B28007800F0825684381402143995089
:1030D0001BE0124A03005BB29B0804246343D258EE
:1030E000FF238407A40F08256C43A3409A4389015A
:1030F000C9B283079B0F0824634399401143074AD1
:1031000040B28008042358431150F0BD14E000E0A1
:1031100018E000E010E000E01CED00E000E400E05A
:1031200080B500203B4908703B480078FD210140F4
:103130003948017000F078F838494018384908607B
:1031400035480078012101433348017001BD10B5B5
:1031500030480478052000F069FB012803D10020E5
:103160002C4908702BE0012000F060FB012803D1FE
:1031700004202849087022E0002000F057FB0128B5
:1031800003D101202349087019E0032000F04EFB11
:10319000012803D102201F49087010E0042000F02C
:1031A00045FB012803D103201A49087007E00220DB
:1031B00000F03CFB012802D1052016490870154893
:1031C0000078E4B2844203D000F02EF8144908607D
:1031D00000F02AF812490968401A1249884206D3B9
:1031E0000D480078FD2101400B48017005E00A48B8
:1031F0000078022101430848017010BD064800789C
:103200000100C9B249080800C007C00F7047014853
:1032100000787047220400202104002018FCFFFFE2
:103220000C040020E90300002A480068704780B5BC
:10323000002009E08100284A891809688022920547
:1032400004234343D150401C3028F3D300F0DCFB6F
:10325000FFF70BFD00F034F8FFF798FCFA21890026
:1032600000F00FFAFFF7FCFE00210020C043FFF73B
:1032700007FF0120FFF75DFD0220FFF75AFD052043
:10328000FFF757FD0323012206211448FFF700FE34
:1032900001BD80B500F0C2FB01BD80B500F0D3FBDD
:1032A00001BD80B5FFF7ACFC01BD7047094800685F
:1032B000401C08490860704700B5FEE7704770473A
:1032C0000748006803218843032101430448016043
:1032D000704700001004002000200008001400487F
:1032E0000000014000203C49087000203B49086074
:1032F00000203B490860704700B501000020C9B2BA
:10330000032905D136490968002902D1012000E0CE
:103310000020C0B200BD00B5062805D0052803D0A6
:10332000072801D0042803D12D490860012003E0BB
:1033300000202B4908600020C0B200BD284800686A
:10334000704725480078704780B5FFF757FF012880
:1033500002D12148007801E0FFF759FFC0B200F028
:1033600069F802BD80B500F041F81B49087001BD45
:103370001A490860704700B5194A1268052A10D129
:10338000000707D515480068802109060143134846
:1033900001601CE011480068400040080F490860C7
:1033A00015E0104A002302400B40002B01D1002AF7
:1033B00007D00A4800688021490501430748016099
:1033C00005E006480068084901400448016000BD66
:1033D0000248006870470000230400201404002005
:1033E0001804002008000200FFFFFFEF00B581076E
:1033F00001D505201CE0002801D1002018E005219E
:103400000140012901D1042012E025210140202999
:1034100001D103200CE07D210140082901D10220C7
:1034200006E07D210140042901D1012000E00620B1
:10343000C0B200BD00B50100C9B2032901D12020EE
:1034400017E00100C9B2022901D1082011E00100F2
:10345000C9B2012901D104200BE00100C9B204293D
:1034600001D1012005E0C0B2052801D1022000E011
:10347000002000BD00B5BFF34F8F2F482F490860D3
:10348000BFF34F8F00BFFDE780B5002000F0FDF9CE
:10349000012809D0002000F034FB012804D00020CE
:1034A000FEF700FF012801D1FFF7E4FF012000F043
:1034B000ECF9012809D0012000F023FB012804D0F9
:1034C0000120FEF7EFFE012806D11D48006801210A
:1034D00001431B48016005E0194800680121884349
:1034E000174908600220FEF7DDFE012806D11448C6
:1034F0000068022101431248016005E0104800689D
:10350000022188430E4908600320FFF7F5FE0128D9
:1035100006D10B480068102101430948016005E00D
:1035200007480068102188430549086001BD044927
:1035300009680840704700000400FA050CED00E03F
:10354000D803002000B500210100C9B230390A2992
:1035500002D23038C0B208E00100C9B241390629B0
:1035600002D23738C0B200E0002000BD0007000FD3
:103570000149085C704700006041000800B5002860
:1035800001D120207CE0C10701D5002078E081072F
:1035900001D5012074E0410701D5022070E0010748
:1035A00001D503206CE0C10601D5042068E0810646
:1035B00001D5052064E0410601D5062060E0010642
:1035C00001D507205CE0C10501D5082058E0810540
:1035D00001D5092054E0410501D50A2050E001053C
:1035E00001D50B204CE0C10401D50C2048E081043A
:1035F00001D50D2044E0410401D50E2040E0010436
:1036000001D50F203CE0C10301D5102038E0810333
:1036100001D5112034E0410301D5122030E001032F
:1036200001D513202CE0C10201D5142028E081022D
:1036300001D5152024E0410201D5162020E0010229
:1036400001D517201CE0C10101D5182018E0810127
:1036500001D5192014E0410101D51A2010E0010123
:1036600001D51B200CE0C10001D51C2008E0810021
:1036700001D51D2004E0400001D51E2000E01F20E0
:1036800000BD0022030A8B420BD203098B4219D2E0
:1036900043088B422ED2411A00D2014652411046B5
:1036A0007047FF2209023FD012068B4205D3121247
:1036B00009028B4201D31212090203098B4219D36A
:1036C00000E0090AC3098B4201D3CB01C01A524161
:1036D00083098B4201D38B01C01A524143098B42AB
:1036E00001D34B01C01A524103098B4201D30B0194
:1036F000C01A5241C3088B4201D3CB00C01A5241B9
:1037000083088B4201D38B00C01A524143088B427D
:1037100001D34B00C01A5241884200D3401A524193
:10372000CFD201461046704708B500F0A1FB08BD96
:1037300080B501220021AD48FFF794FB01220A2148
:10374000AA48FFF78FFB01220B21A848FFF78AFB4D
:1037500001220D21A548FFF785FB01220E21A34878
:10376000FFF780FB01220F21A048FFF77BFBFFF74B
:103770005BFD0A389E49086000209E4908609E480B
:103780000078012101439C4801709B480078FB218F
:1037900001409948017098480078FD210140964801
:1037A000017001BD10B5944800780100C907C90F28
:1037B000002934D091480468FFF736FD8C49096828
:1037C000401A0A281ED38D480468FFF72DFD88494A
:1037D000086000F07DF800F0D6F888490860874856
:1037E000006800F0AFF8002806D183480078042173
:1037F00001438148017005E07F480078FB210140CA
:103800007D4801707D48006860407D4908607C48C3
:1038100000687A49096801407948016005E0764806
:103820000078022101437448017010BD00B5010009
:10383000C9B2052901D120201DE00100C9B201292A
:1038400001D1022017E00100C9B2002901D10120F5
:1038500011E00100C9B2032901D108200BE00100E9
:10386000C9B2042901D1102005E0C0B2022801D15B
:10387000042000E00020614909680840002801D0C8
:10388000012000E00020C0B200BD00B50100002012
:103890000A00D2B2012A0AD157490978C9B2890867
:1038A0000A00D207D20F002A10D001200EE0C9B2C0
:1038B00000290AD150490978C9B249080A00D2073B
:1038C000D20F002A02D0012000E00020C0B200BDCB
:1038D00010B5002400214548FFF780FB002802D1E5
:1038E0002000012404430A214048FFF777FB002809
:1038F00002D12000022404430B213C48FFF76EFB59
:10390000002802D12000042404430D213748FFF78A
:1039100065FB002802D12000082404430E2133480F
:10392000FFF75CFB002802D12000102404430F2184
:103930002E48FFF753FB002802D120002024044327
:10394000200010BD00B50100012000290BD008297E
:1039500014D0102912D0202910D001290ED002290C
:103960000CD004290AD023490968491C214A116056
:10397000204909680A2904D3002002E000211D4AD9
:103980001160C0B200BD30B501000A00002006E0A1
:1039900014001C4A04234343D2582243401C0328EA
:1039A000F6D31848C06802400800002306E005006E
:1039B000144804245C43005928405B1C032BF6D3B5
:1039C0001043104AD06002220AE00E4B04245443F4
:1039D0001B191B1F1B680B4C042555436351521EBA
:1039E000002AF2D1074A116030BD000000040048EF
:1039F000F8030020FC0300201F040020F003002037
:103A0000F4030020C803002003480068102101438C
:103A100001480160704700000020024000B50C48DA
:103A20000C4908600C480B49086000200B490860ED
:103A30000B480C4908600C4800680028FBD10B4873
:103A40000449086000BD0948024908607047000049
:103A5000CCCC000000300040555500000430004040
:103A6000FF0F0000083000400C300040AAAA000000
:103A700080B50023012200219020C005FFF708FA3D
:103A80000023012201219020C005FFF701FA002345
:103A9000012202219020C005FFF7FAF9002301223C
:103AA00003219020C005FFF7F3F900230122042130
:103AB0009020C005FFF7ECF9002200219020C005FE
:103AC000FFF77FFA002201219020C005FFF779FA65
:103AD000002202219020C005FFF773FA0022032183
:103AE0009020C005FFF76DFA002204219020C00548
:103AF000FFF767FAB548007801210143B348017028
:103B000001BD00B501000020C9B200290AD1AF49AA
:103B10000978C9B2C9080A00D207D20F002A02D018
:103B2000012000E00020C0B200BD80B50120FFF7F9
:103B3000FEFC002803D01F2000F0BAF8B7E00220F6
:103B4000FFF7F5FC002804D11020FFF7F0FC002857
:103B50001CD0FFF769FB9E490968401AC82800D2AB
:103B6000A5E0FFF761FB9A49086098480078C0B269
:103B700040080100C907C90F002903D0002000F048
:103B800097F894E01F2000F093F890E0FFF720FCF6
:103B9000002865D0FEF7A9FB002861D1FFF72EFBB6
:103BA00000285DD189480078C0B280080100C907AB
:103BB000C90F002928D0FFF737FB85490968401A4B
:103BC000C82826D381480078C0B240080100C90740
:103BD000C90F002909D0002000F06AF87B4800785E
:103BE000FD2101407948017009E09A48006800F021
:103BF0005FF8764800780221014374480170FFF7AE
:103C000013FB7349086004E0FFF79BFBC0B200F0B0
:103C10009DF8FFF709FB90490968401A8F498842CF
:103C200045D36A480078C0B280080100C907C90FAF
:103C3000002906D065480078FB21014063480170E7
:103C400009E062480078042101436048017000F0F7
:103C5000C1F880490860FFF7E7FA7F49086026E06D
:103C6000FEF743FB012803D0FFF7C8FA01280FD164
:103C7000FFF7CDFAC0B200F069F85448007804218B
:103C8000014352480170FFF7CFFA734908600EE014
:103C9000FFF757FBC0B200F059F84C4800780421F8
:103CA00001434A480170FFF7BFFA6B49086001BD44
:103CB00010B50400E00606D4002200219020C005C3
:103CC000FFF77FF905E0012200219020C005FFF7F2
:103CD00078F9600706D4002202219020C005FFF782
:103CE00070F905E0012202219020C005FFF769F973
:103CF000200706D4002201219020C005FFF761F9BA
:103D000005E0012201219020C005FFF75AF9E007E4
:103D100006D4002204219020C005FFF752F905E0E7
:103D2000012204219020C005FFF74BF9A00706D41B
:103D3000002203219020C005FFF743F905E001228E
:103D400003219020C005FFF73CF910BD80B50100AC
:103D5000C9B2002903D10420FFF7AAFF34E0010013
:103D6000C9B2022903D10120FFF7A2FF2CE0010014
:103D7000C9B2012903D10820FFF79AFF24E001000E
:103D8000C9B2042903D11020FFF792FF1CE0010003
:103D9000C9B2032903D10220FFF78AFF14E0010012
:103DA000C9B2052903D10020FFF782FF0CE0C0B2A1
:103DB000062803D11820FFF77BFF05E003480078B1
:103DC000102101430148017001BD000020040020C2
:103DD0000404002010B5FFF7FBFA002100E0491CA5
:103DE000202917D21E4A126880235B059A4209D007
:103DF0001B4A1268002A05D0194A12685200184B53
:103E00001A6002E00122164B1A60154A126802403D
:103E1000002AE4D012480068FFF7B0FB0400202C11
:103E200016D2FFF78BFA062804D10E4804214C4322
:103E300000590EE0FFF782FA052804D10A48042150
:103E40004C43005905E0094804214C43005900E067
:103E5000002010BD0004002008040020B80B000062
:103E6000C0000020F43E0008743F0008743E0008C3
:103E70007047FEE70D0000000D0000000400000088
:103E80000D000000010000000F000000070000000E
:103E900008000000020000000A0000000B00000003
:103EA0000B000000110000000B0000000E000000DD
:103EB00010000000030000001200000013000000CA
:103EC0000B000000050000001600000018000000B4
:103ED0001A0000000D0000001B0000000D00000093
:103EE0001D00000009000000180000000200000092
:103EF0001F0000000D0000000D0000000400000085
:103F00000D000000010000000F000000070000008D
:103F100008000000020000000A0000000B00000082
:103F20000B0000000B0000000B0000000E00000062
:103F30001000000003000000120000001300000049
:103F40000B00000005000000160000001800000033
:103F50001A0000000D0000001B0000000D00000012
:103F60001D00000009000000180000000200000011
:103F70001F0000000100000001000000040000001C
:103F80000D00000001000000070000000A00000012
:103F90000B0000000B0000000E00000010000000ED
:103FA00012000000130000000B00000016000000CB
:103FB00018000000180000001A0000001B0000009C
:103FC00006000000060000000600000006000000D9
:103FD000060000000F0000001D0000001D00000092
:103FE00011000000020000000D0000000D000000A4
:103FF0000900000070B40123002413E00168001DD3
:10400000194202D04D466D1E49190C60091D121F40
:10401000042AFAD20D00960701D50C80AD1C1A4077
:1040200000D02C700268001D002AE7D170BC7047D8
:1040300080B5FFF7FCF8FFF755F9FEF74CF8FFF7EE
:1040400077FBFFF715FDFFF76BF8FFF722F9FFF796
:1040500024F9FFF7A7FBFFF77AF8FEF7C7F8FFF799
:1040600064FDFFF711FAF2E730B401220168001D88
:1040700000290FD00368C31844680830144202D0E6
:104080004D466D1E64191D6825601B1D241D091FEA
:10409000ECD0F8E730BC704710B5074979441831C7
:1040A000064C7C44163404E0081D0A6889188847C9
:1040B0000100A142F8D110BD080000002800000056
:1040C00035FFFFFF5C030000C80000200000000077
:1040D00099FFFFFF08000000B4000000C0000020AE
:1040E0000000000000F00DF8002801D0FFF7D4FF19
:1040F00000BF00BF002000BF00BFFFF799FF00F026
:1041000002F80120704780B500F002F801BDFEE71B
:104110000746384600F002F8FBE7FEE780B500BF2F
:1041200000BF024A11001820ABBEFBE726000200C8
:10413000000000000102030401020304060708094D
:1041400002030405060708090A0B0C0D0E0F1010D8
:104150000102030405060708090A0B0C0D0E0F10D7
:1041600030313233343536373839414243444546AD
:104170000148804701480047A332000881410008F8
:1041800000BF00BF00BF00BFFFF7ACFF0100000091
:1041900000127A00FEE7FEE7FEE7FEE7FEE7FEE735
:1041A000FEE7FEE7FEE7FEE7FEE7FEE7FEE7FEE7E7
:0A41B000FEE7FEE7FEE7FEE7FEE78C
:04000005080041812D
:00000001FF
